:020000040000FA
:0A0000000000000049EF01F05ED19E
:08001800B1D19EA8FED7AD6E28
:1000200012000C6A0B6EFF0E0B260C2200D0D8A01B
:100030001200030E0A6EE60E02D8F5D70A6AFE0F0A
:10004000096EE86A0A5AD8A012000000090600D01A
:10005000F8D71450105C196E11E2196C105014C0CE
:1000600010F0146E115015C011F0156E125016C01C
:1000700012F0166E135017C013F0176E1A0E196097
:1000800074D0145272E0186A11501C6E15181B6E51
:10009000118E158E080E195E08E317C018F016C0F1
:1000A00017F015C016F0156AF5D7192607E0D89095
:1000B0001532163217321832192EF9D71BAE33D03B
:1000C0001750135E1650125A1550115A07E2D88075
:1000D000000E135612561156800E1C1A186C04E0AE
:1000E0001306000E125A115A040E196E11660DD025
:1000F00012C011F013C012F018C013F0186A080EE5
:10010000105E29E3192EF2D726D011BE08D0D89060
:100110001836133612361136102EF7D71CD018AEFB
:1001200022D0186A0FD017501326165012221550DD
:10013000112206E31132123213321832104A0DD056
:1001400018AE11D0133E0FD0123E0DD0113E0BD081
:10015000D8801390EFD7106A02D01A821068136A01
:10016000126A800E116E1CAE119E1350120010C048
:100170001CF0115013C011F0136E13361C321332E1
:100180001A6A13361C3602E31A841A7E06E11A80B4
:100190001C6A136A126A116A0BD01C2803E0D8800B
:1001A000133206D0D890133202E11A8201D01A8697
:1001B0001AB604D01AA20FD01AB407D07F0E136E4D
:1001C000FF0E126E116E106E23D0800E136E01D0D2
:1001D000136A000EF6D71AB0FBD7106A9F0E1C6088
:1001E000EBD77E0E1C64F4D79E0E1C5C07E0D89003
:1001F00013321232113210321C2AF6D71AA408D048
:10020000D880000E105611561256135613AEE0D772
:1002100010501200126A136A1B9E0AD01B9E13AE66
:1002200007D0D880000E10561156125613561B8E4A
:10023000960E1C6E135209E0080E1C2611C010F019
:1002400012C011F013C012F011D012520FE1080EBB
:100250001C5E115007E1080E1C5E105002E11350A5
:1002600010D0106A126E10C011F0106A12BE06D0C3
:10027000D8901036113612361C06F8D71BAE129ED7
:100280001C5010C013F0106E125011C012F0116EFD
:100290001200400E1A6E006A4F0EAF6EB06A240E46
:1002A000AC6E900EAB6E00010F0EC16E070EB46EF9
:1002B000C69AC00E926EE00E936EC00E946E956A52
:1002C000E80E966E70D0F2A409D0F294244A252A42
:1002D000D6CF22F0D7CF23F0817A11009EAA19D071
:1002E000060EAB1412E1E2CF1FF0E1CF1EF0202A80
:1002F00010EE6EF02050E126000EE222AECFE7FFB6
:100300001FC0E2FF1EC0E1FF1100AE50AE50AB981F
:10031000AB8811002050215C14E0212AEACF0AF0BA
:10032000E9CF09F000EE6EF02150E926000EEA2236
:10033000EF501D6E0AC0EAFF09C0E9FFD880120025
:1003400004D0E8681D6ED8A012001200206A216A4D
:100350009D8A9F8AF28EF28C12009D9A00EE6EF0BA
:10036000010EF46EF36AF306000EF45AEE6AF450CE
:10037000F310F9E1206A216A9D8A1200F29EE0CF13
:10038000EEF3D8CFEFF3E8CFF0F3F28E0001A192B5
:10039000B36AB26AF29EEEC3E0FFEFC3D8FFF0C3C8
:1003A000E8FFF28E1000939A8A9A0A0E3ADE929231
:1003B000899292968996929A899A96928D9293981A
:1003C0008A9893948A9493908A90959C8C9C959803
:1003D0008C9894988B9895948C9494928B929496F4
:1003E0008B9695928C9292948994929089909298FF
:1003F000899896908D9096948D9493968A969392E0
:100400008A92959E8C9E959A8C9A949A8B9A9596A0
:100410008C9694908B9094948B9495908C9000EE05
:1004200049F0200EEE68E82EFDD73968280E366EAA
:10043000456A446A8BDF91DFCD6AF294F28A870EB7
:10044000D56EB16AA192A082D08EA292B10EB16E89
:10045000C0EC07F0E2EC09F007EC13F033500DECC0
:1004600000F0420E0DEC00F0400E0DEC00F0D6CF87
:1004700022F0D7CF23F04EDF1DC02AF0BE0E2A5C3B
:1004800007E3FE0E2A5C01E301D02C6A52EF06F06E
:100490002AAE22D02C6A8D0E2A5C05E12AC02CF0EF
:1004A0002D682E6817D09D0E2A5C05E12AC02CF01D
:1004B0002F6830680FD0AD0E2A5C05E12AC02CF001
:1004C0003168326807D0BD0E2A5C04E12AC02CF0E6
:1004D0003368346851EF06F02C5204E152EF06F015
:1004E00051EF06F08D0E2C5CD8A40AD12D2803E123
:1004F0002AC02DF001D12AC02EF0300E2D5CD8A0DC
:1005000041D05E0E2D5CD8B03DD02D50475C39E116
:10051000476AFF0E2224026EFF0E2320036E000E98
:100520002420046E000E2520056E05C04CF004C08A
:100530004BF003C04AF002C049F02DC048F0899248
:100540008996899A8D928A988A948A908C9C506810
:100550004F684E684D68392814E1000E2224026E5F
:10056000200E2320036E000E2420046E000E252092
:10057000056E05C068F004C067F003C066F002C0F5
:1005800065F0B7D05E0E2D5CD8A43ED02D50475CF0
:100590003AE1476AFF0E2224026EFF0E2320036E0B
:1005A000000E2420046E000E2520056E05C04CF0C0
:1005B00004C04BF003C04AF002C049F02DC048F01F
:1005C00089928996899A8D928A988A948A908C9C2D
:1005D0008C9850684F684E684D68392814E1000EB9
:1005E0002224026E200E2320036E000E2420046EAF
:1005F000000E2520056E05C068F004C067F003C03A
:1006000066F002C065F075D05F0E2D5CD8A041D0B9
:100610006A0E2D5CD8B03DD02D50475C39E1476A59
:10062000FF0E2224026EFF0E2320036E000E2420F4
:10063000046E000E2520056E05C04CF004C04BF082
:1006400003C04AF002C049F02DC048F08992899653
:10065000899A8D928A988A948A908C9C50684F6867
:100660004E684D68392814E1000E2224026E200ED7
:100670002320036E000E2420046E000E2520056E3C
:1006800005C068F004C067F003C066F002C065F002
:1006900030D0780E2D5C06E154685368526851687A
:1006A0008B9A27D0790E2D5C06E18C965868576896
:1006B000566855681ED07A0E2D5C06E18B905C68FA
:1006C0005B685A68596815D07B0E2D5C08E1395279
:1006D00005E18B9460685F685E685D680AD07C0E97
:1006E0002D5C07E1395205E18C90646863686268AB
:1006F00061682D6851EF06F052EF06F051EF06F0F9
:100700009D0E2C5CD8A436EF06F02F2804E12AC0F9
:100710002FF034EF06F02AC030F03052D8A402D1C6
:10072000300E2F5CD8A041D05E0E2F5CD8B03DD0EB
:100730002F50475C39E1476AFF0E2224026EFF0EFC
:100740002320036E000E2420046E000E2520056E6B
:1007500005C04CF004C04BF003C04AF002C049F0A1
:100760002FC048F089928996899A8D928A988A94A6
:100770008A908C9C50684F684E684D68392814E107
:10078000000E2224026E200E2320036E000E242071
:10079000046E000E2520056E05C068F004C067F0E9
:1007A00003C066F002C065F0BAD05E0E2F5CD8A41C
:1007B0003ED02F50475C3AE1476AFF0E2224026E7A
:1007C000FF0E2320036E000E2420046E000E252051
:1007D000056E05C04CF004C04BF003C04AF002C0E7
:1007E00049F02FC048F089928996899A8D928A980B
:1007F0008A948A908C9C8C9850684F684E684D689B
:10080000392814E1000E2224026E200E2320036EEC
:10081000000E2420046E000E2520056E05C068F031
:1008200004C067F003C066F002C065F078D05F0EC8
:100830002F5CD8A041D06A0E2F5CD8B03DD02F508D
:10084000475C39E1476AFF0E2224026EFF0E232027
:10085000036E000E2420046E000E2520056E05C0D8
:100860004CF004C04BF003C04AF002C049F02FC066
:1008700048F089928996899A8D928A988A948A906A
:100880008C9C50684F684E684D68392814E1000E02
:100890002224026E200E2320036E000E2420046EFC
:1008A000000E2520056E05C068F004C067F003C087
:1008B00066F002C065F033D0780E2F5C06E1546814
:1008C0005368526851688B9A2AD0790E2F5C06E1E2
:1008D00058685768566855688C9621D07A0E2F5CF8
:1008E00006E15C685B685A6859688B9018D07B0E8B
:1008F0002F5C08E1395205E160685F685E685D68F9
:100900008B940DD07C0E2F5C08E1395205E16468B0
:100910006368626861688C9002D02F68C3D12F68C9
:10092000C0D1A2D1300E2F5CD8A07ED06A0E2F5C31
:10093000D8B07AD04C684B684A68496803EE6EF0CC
:100940002F50EB50466E03EE6EF04850EB502B6E7E
:1009500046B002D0899403D089842BA0898246B204
:1009600002D0899003D089802BA2898646B402D018
:10097000899803D089882BA4898A46B602D08D90A5
:1009800003D08D802BA68D8246B802D08D9403D0E3
:100990008D842BA88A8846BA02D08A9603D08A868C
:1009A0002BAA8A8446BC02D08A9203D08A822BACBE
:1009B0008A8046BE02D08C9E03D08C8E2BAE8C8C4F
:1009C0005E0E2F5C06E18C8A5E0E485C01E08C882E
:1009D00001D08C9A392806E168686768666865689E
:1009E0008B848C802FC047F001EE6EF0D8903634A7
:1009F000E926000EEA22EECF44F0EFCF45F0445056
:100A00002224026E45502320036E000E2420046E23
:100A1000000E2520056E05C050F004C04FF003C045
:100A20004EF002C04DF01ED1780E2F5C35E17F0EE6
:100A3000305C2CE28B8A02EE6EF0D8903034E926DE
:100A4000000EEA22EECF06F0EFCF07F00650222488
:100A5000026E07502320036E000E2420046E000E49
:100A60002520056E05C054F004C053F003C052F0B9
:100A700002C051F002EE6EF0D8903034E926000E3C
:100A8000EA22EECF3AF0EFCF3BF005D08B8A5468E4
:100A9000536852685168E6D0790E2F5C35E17F0EBD
:100AA000305C2CE28C8602EE6EF0D8903034E92671
:100AB000000EEA22EECF06F0EFCF07F00650222418
:100AC000026E07502320036E000E2420046E000ED9
:100AD0002520056E05C058F004C057F003C056F03D
:100AE00002C055F002EE6EF0D8903034E926000EC8
:100AF000EA22EECF3CF0EFCF3DF005D08C8658686F
:100B0000576856685568AED07A0E2F5C35E17F0E77
:100B1000305C2CE28B8002EE6EF0D8903034E92607
:100B2000000EEA22EECF06F0EFCF07F006502224A7
:100B3000026E07502320036E000E2420046E000E68
:100B40002520056E05C05CF004C05BF003C05AF0C0
:100B500002C059F002EE6EF0D8903034E926000E53
:100B6000EA22EECF3EF0EFCF3FF005D08B805C68FD
:100B70005B685A68596876D07B0E2F5C37E1395232
:100B800034E17F0E305C2CE28B8402EE6EF0D89064
:100B90003034E926000EEA22EECF06F0EFCF07F060
:100BA00006502224026E07502320036E000E2420DC
:100BB000046E000E2520056E05C060F004C05FF0D5
:100BC00003C05EF002C05DF002EE6EF0D8903034EB
:100BD000E926000EEA22EECF40F0EFCF41F005D03B
:100BE0008B8460685F685E685D683CD07C0E2F5CBB
:100BF00037E1395234E17F0E305C2CE28C8002EE1A
:100C00006EF0D8903034E926000EEA22EECF06F0DE
:100C1000EFCF07F006502224026E07502320036E08
:100C2000000E2420046E000E2520056E05C064F021
:100C300004C063F003C062F002C061F002EE6EF027
:100C4000D8903034E926000EEA22EECF42F0EFCF02
:100C500043F005D08C80646863686268616802D084
:100C60002F6820D02F681DD01DD01BD0AD0E2C5C5E
:100C70000AE1312803E12AC031F003D02AC032F062
:100C80000BD910D00ED0BD0E2C5C0AE1332803E145
:100C90002AC033F003D02AC034F000D903D001D0E9
:100CA00001D0C0D8080E6D5CD8B0B6D06950225CB7
:100CB0006A5023586B5024586C502558D8A0ABD09C
:100CC0006C8E6D5210E18994899089988D908D94E5
:100CD0008A968A928C9E8C9A466A4C684B684A68BF
:100CE0004968486A97D0010E6D5C0EE18992899639
:100CF000899A8D928A988A948A908C9C8C98506854
:100D00004F684E684D6886D0020E6D5C16E1827A9F
:100D10003A502224026E3B502320036E000E242002
:100D2000046E000E2520056E05C054F004C053F07B
:100D300003C052F002C051F06DD0030E6D5C16E19D
:100D400083763C502224026E3D502320036E000E19
:100D50002420046E000E2520056E05C058F004C046
:100D600057F003C056F002C055F054D0040E6D5C2D
:100D700016E182703E502224026E3F502320036E03
:100D8000000E2420046E000E2520056E05C05CF0C8
:100D900004C05BF003C05AF002C059F03BD0050E0E
:100DA0006D5C16E1827440502224026E4150232073
:100DB000036E000E2420046E000E2520056E05C073
:100DC00060F004C05FF003C05EF002C05DF022D0AE
:100DD000060E6D5C16E1837042502224026E435071
:100DE0002320036E000E2420046E000E2520056EC5
:100DF00005C064F004C063F003C062F002C061F09B
:100E000009D0070E6D5C06E168686768666865680A
:100E10008B948C9007D804D025AE02D0256A246A22
:100E200037EF02F06D686C8E2B6A080E2B5C33E294
:100E3000D8902B34E96EEA6AEA36E936EA36490E8A
:100E4000E926000EEA22EFCF02F0ECCF03F0ECCF60
:100E500004F0ECCF05F06950025C6A5003586B5007
:100E600004586C50055815E2D8902B34E96EEA6AA4
:100E7000EA36E936EA36490EE926000EEA22EFCFD5
:100E800069F0ECCF6AF0ECCF6BF0ECCF6CF02BC0DC
:100E90006DF02B2ACAE3120031681200190E335C80
:100EA00003E134C036F042D0420E335C09E13452E3
:100EB00002E13ED804D039683768280E366E36D045
:100EC000450E335C0DE1400E345C08E28B948C904F
:100ED0006868676866686568396A01D0396826D0CD
:100EE0007B0E335C23E100EE49F0200EEE68E82E25
:100EF000FDD789928996899A8D928A988A948A9048
:100F00008C9C8C988B988C948B928B968C928994D9
:100F1000899089988D908D948A968A928C9E8C9ACD
:100F20008B9A8C968B908B948C907CDF336812001C
:100F3000386A00EE49F0200EEE68E82EFDD73968D9
:100F4000376A280E366E89928996899A8D928A9888
:100F50008A948A908C9C8C988B988C948B928B968C
:100F60008C928994899089988D908D948A968A9292
:100F70008C9E8C9A8B9A8C968B908B948C9052D75B
:100F800002016F696E695C0E716F7A0E706F590E97
:100F9000736F850E726F580E756F140E746F560E48
:100FA000776FA90E766F550E796F430E786F530EDB
:100FB0007B6FE30E7A6F520E7D6F890E7C6F510E40
:100FC0007F6F350E7E6F4F0E816FE60E806F4E0E77
:100FD000836F9C0E826F4D0E856F580E846F4C0E82
:100FE000876F190E866F4A0E896FDF0E886F490E64
:100FF0008B6FAA0E8A6F480E8D6F7A0E8C6F470E1C
:101000008F6F4F0E8E6F460E916F290E906F450EAB
:10101000936F080E926F430E956FEB0E946F420E16
:10102000976FD30E966F410E996FBF0E986F400E5B
:101030009B6FB00E9A6F3F0E9D6FA50E9C6F3E0E7C
:101040009F6F9E0E9E6F3D0EA16F9C0EA06F3C0E7B
:10105000A36F9E0EA26F3B0EA56FA40EA46F3A0E57
:10106000A76FAE0EA66F390EA96FBC0EA86F380E13
:10107000AB6FCE0EAA6F370EAD6FE30EAC6F360EB0
:10108000AF6FFD0EAE6F360EB16F1A0EB06F350E2C
:10109000B36F3B0EB26F340EB56F5F0EB46F330E8D
:1010A000B76F870EB66F320EB96FB20EB86F310ED2
:1010B000BB6FE10EBA6F310EBD6F140EBC6F300EF8
:1010C000BF6F490EBE6F2F0EC16F820EC06F2E0E06
:1010D000C36FBE0EC26F2D0EC56FFD0EC46F2D0EF9
:1010E000C76F3F0EC66F2C0EC96F850EC86F2B0ED3
:1010F000CB6FCD0ECA6F2B0ECD6F180ECC6F2A0E94
:10110000CF6F670ECE6F290ED16FB80ED06F290E3C
:10111000D36F0C0ED26F280ED56F620ED46F270ED0
:10112000D76FBC0ED66F270ED96F180ED86F260E4C
:10113000DB6F760EDA6F250EDD6FD80EDC6F250EB5
:10114000DF6F3C0EDE6F240EE16FA20EE06F240E07
:10115000E36F0B0EE26F230EE56F760EE46F220E47
:10116000E76FE40EE66F220EE96F540EE86F210E72
:10117000EB6FC60EEA6F210EED6F3B0EEC6F200E8B
:10118000EF6FB20EEE6F200EF16F2B0EF06F1F0E91
:10119000F36FA60EF26F1F0EF56F240EF46F1E0E86
:1011A000F76FA30EF66F1E0EF96F250EF86F1D0E6A
:1011B000FB6FA90EFA6F1D0EFD6F2E0EFC6F1C0E3D
:1011C000FF6FB60EFE6F1C0E0301016F3F0E006F26
:1011D0001B0E036FCB0E026F1B0E056F580E046FB4
:1011E0001A0E076FE80E066F1A0E096F790E086F58
:1011F0001A0E0B6F0B0E0A6F190E0D6FA00E0C6FEF
:10120000190E0F6F360E0E6F180E116FCE0E106F77
:10121000180E136F680E126F180E156F030E146FF1
:10122000170E176FA00E166F170E196F3F0E186F5F
:10123000160E1B6FDF0E1A6F160E1D6F800E1C6FC1
:10124000160E1F6F240E1E6F150E216FC80E206F15
:10125000150E236F6E0E226F150E256F160E246F5E
:10126000140E276FBF0E266F140E296F690E286F9C
:10127000140E2B6F150E2A6F130E2D6FC20E2C6FCE
:10128000130E2F6F710E2E6F130E316F210E306FF4
:10129000120E336FD20E326F120E356F840E346F12
:1012A000120E376F380E366F110E396FED0E386F24
:1012B000110E3B6FA30E3A6F110E3D6F5A0E3C6F2D
:1012C000110E3F6F120E3E6F100E416FCC0E406F2D
:1012D000100E436F870E426F100E456F420E446F23
:1012E0000F0E476F4669496FBD0E486F0F0E4B6F6B
:1012F0007C0E4A6F0F0E4D6F3D0E4C6F0E0E4F6FF2
:10130000FE0E4E6F0E0E516FC00E506F0E0E536FCD
:10131000830E526F0E0E556F470E546F0E0E576FA1
:101320000C0E566F0D0E596FD20E586F0D0E5B6F6F
:10133000990E5A6F0D0E5D6F610E5C6F0D0E5F6F33
:101340002A0E5E6F0C0E616FF40E606F0C0E636FF1
:10135000BE0E626F0C0E656F8A0E646F0C0E676FA7
:10136000560E666F0C0E696F230E686F0B0E6B6F57
:10137000F10E6A6F0B0E6D6FC00E6C6F010E2B6E4F
:101380000001800E2B5C1DE202EE6EF0D8902B3433
:10139000E926000EEA22EECF06F0EFCF07F0D89054
:1013A0000730036E0630026E02EE6EF0D8902B34DA
:1013B000E926000EEA2202C0EEFF03C0EFFF2B2A4F
:1013C000DFE312000101716B340E706F020E2B6EA1
:1013D0000001800E2B5C36E22B04086E01EE6EF0ED
:1013E000D8900834E926000EEA22EECF06F0EFCFBF
:1013F00007F006C010F007C011F00AEC01F013C0AE
:1014000017F012C016F011C015F010C014F0330E12
:10141000136E126E030E116E840E106E29EC00F026
:10142000B7EC00F0026E11C003F001EE6EF0D89040
:101430002B34E926000EEA2202C0EEFF03C0EFFFC4
:101440002B2AC6E3010E2B6E800E2B5C1DE201EEF3
:101450006EF0D8902B34E926000EEA22EECF06F08B
:10146000EFCF07F0D8900730036E0630026E01EE22
:101470006EF0D8902B34E926000EEA2202C0EEFF6F
:1014800003C0EFFF2B2AE0E312000101716B340E61
:10149000706F736B380E726F756B3A0E746F776B7B
:1014A0003C0E766F796B3E0E786F7B6B400E7A6FD9
:1014B0007D6B420E7C6F7F6B450E7E6F816B470E9E
:1014C000806F836B490E826F856B4C0E846F876BC8
:1014D0004F0E866F896B510E886F8B6B540E8A6F1F
:1014E0008D6B570E8C6F8F6B5A0E8E6F916B5E0EDD
:1014F000906F936B610E926F956B640E946F976B08
:10150000680E966F996B6B0E986F9B6B6F0E9A6F50
:101510009D6B730E9C6F9F6B770E9E6FA16B7B0E06
:10152000A06FA36B800EA26FA56B840EA46FA76B38
:10153000890EA66FA96B8E0EA86FAB6B930EAA6F68
:10154000AD6B980EAC6FAF6B9D0EAE6FB16BA30E13
:10155000B06FB36BA80EB26FB56BAE0EB46FB76B56
:10156000B40EB66FB96BBB0EB86FBB6BC10EBA6F62
:10157000BD6BC80EBC6FBF6BCF0EBE6FC16BD60EFE
:10158000C06FC36BDE0EC26FC56BE60EC46FC76B58
:10159000EE0EC66FC96BF60EC86FCB6BCA69010E33
:1015A000CD6F080ECC6F010ECF6F110ECE6F010EF6
:1015B000D16F1B0ED06F010ED36F250ED26F010EAF
:1015C000D56F2F0ED46F010ED76F3A0ED66F010E66
:1015D000D96F450ED86F010EDB6F500EDA6F010E1A
:1015E000DD6F5C0EDC6F010EDF6F680EDE6F010ECB
:1015F000E16F750EE06F010EE36F820EE26F010E78
:10160000E56F900EE46F010EE76F9E0EE66F010E20
:10161000E96FAC0EE86F010EEB6FBB0EEA6F010EC7
:10162000ED6FCB0EEC6F010EEF6FDB0EEE6F010E68
:10163000F16FEC0EF06F010EF36FFD0EF26F020E04
:10164000F56F0F0EF46F020EF76F210EF66F020E9C
:10165000F96F340EF86F020EFB6F480EFA6F020E30
:10166000FD6F5D0EFC6F020EFF6F720EFE6F020EBD
:101670000201016F880E006F020E036F9F0E026F52
:10168000020E056FB70E046F020E076FCF0E066FC6
:10169000020E096FE80E086F030E0B6F020E0A6F41
:1016A000030E0D6F1E0E0C6F030E0F6F3A0E0E6FB2
:1016B000030E116F570E106F030E136F750E126F1E
:1016C000030E156F940E146F030E176FB40E166F82
:1016D000030E196FD50E186F030E1B6FF80E1A6FDD
:1016E000040E1D6F1C0E1C6F040E1F6F410E1E6F2B
:1016F000040E216F670E206F040E236F8E0E226F73
:10170000040E256FB70E246F040E276FE20E266FAE
:10171000050E296F0E0E286F050E2B6F3B0E2A6FDC
:10172000050E2D6F6A0E2C6F050E2F6F9B0E2E6F00
:10173000050E316FCE0E306F060E336F020E326F14
:10174000060E356F380E346F060E376F700E366F1B
:10175000060E396FAA0E386F060E3B6FE60E3A6F13
:10176000070E3D6F240E3C6F070E3F6F640E3E6FF9
:10177000070E416FA70E406F070E436FEC0E426FCE
:10178000080E456F330E446F080E476F7D0E466F8F
:10179000080E496FC90E486F090E4B6F180E4A6F3D
:1017A000090E4D6F6A0E4C6F090E4F6FBF0E4E6FD4
:1017B0000A0E516F170E506F0A0E536F720E526F52
:1017C0000A0E556FD00E546F0B0E576F310E566FB9
:1017D0000B0E596F960E586F0B0E5B6FFE0E5A6F05
:1017E0000C0E5D6F6A0E5C6F0C0E5F6FDA0E5E6F33
:1017F0000D0E616F4D0E606F0D0E636FC50E626F43
:101800000E0E656F410E646F0E0E676FC10E666F30
:101810000F0E696F460E686F0F0E6B6FD00E6A6FFA
:10182000100E6D6F5E0E6C6F010E2B6E0001800E40
:101830002B5C1DE201EE6EF0D8902B34E926000EF1
:10184000EA22EECF06F0EFCF07F0D8900730036E14
:101850000630026E01EE6EF0D8902B34E926000EB1
:10186000EA2202C0EEFF03C0EFFF2B2ADFE31200E3
:101870000101716B2F0E706F020E2B6E0001800E36
:101880002B5C20E22B04086E01EE6EF0D890083439
:10189000E926000EEA22EECF06F0EFCF07F0140E95
:1018A0000624026E000E0720036E01EE6EF0D89043
:1018B0002B34E926000EEA2202C0EEFF03C0EFFF40
:1018C0002B2ADCE3010E2B6E800E2B5C1DE201EE59
:1018D0006EF0D8902B34E926000EEA22EECF06F007
:1018E000EFCF07F0D8900730036E0630026E01EE9E
:1018F0006EF0D8902B34E926000EEA2202C0EEFFEB
:1019000003C0EFFF2B2AE0E312000101716B2E0EE2
:10191000706F020E2B6E0001800E2B5C37E22B04E1
:10192000086E01EE6EF0D8900834E926000EEA2227
:10193000EECF06F0EFCF07F006C010F007C011F0B1
:101940000AEC01F013C017F012C016F011C015F028
:1019500010C014F00A0E136ED70E126E470E116EE1
:10196000820E106E29EC00F0B7EC00F0026E11C090
:1019700003F001EE6EF0D8902B34E926000EEA2237
:1019800002C0EEFF03C0EFFF2B2AC5E3010E2B6E52
:10199000800E2B5C1DE201EE6EF0D8902B34E92610
:1019A000000EEA22EECF06F0EFCF07F0D890073016
:1019B000036E0630026E01EE6EF0D8902B34E926ED
:1019C000000EEA2202C0EEFF03C0EFFF2B2AE0E385
:1019D00012000101716B2F0E706F736B320E726FFC
:1019E000756B340E746F776B350E766F796B370EBF
:1019F000786F7B6B390E7A6F7D6B3B0E7C6F7F6BE4
:101A00003C0E7E6F816B3E0E806F836B400E826F4B
:101A1000856B420E846F876B450E866F896B470E10
:101A2000886F8B6B490E8A6F8D6B4B0E8C6F8F6B33
:101A30004E0E8E6F916B500E906F936B530E926F94
:101A4000956B560E946F976B580E966F996B5B0E55
:101A5000986F9B6B5E0E9A6F9D6B610E9C6F9F6B78
:101A6000640E9E6FA16B670EA06FA36B6B0EA26FCF
:101A7000A56B6E0EA46FA76B720EA66FA96B750E89
:101A8000A86FAB6B790EAA6FAD6B7D0EAC6FAF6BB1
:101A9000810EAE6FB16B850EB06FB36B890EB26FF6
:101AA000B56B8E0EB46FB76B920EB66FB96B970EA7
:101AB000B86FBB6B9C0EBA6FBD6BA10EBC6FBF6BDA
:101AC000A60EBE6FC16BAB0EC06FC36BB10EC26F03
:101AD000C56BB60EC46FC76BBC0EC66FC96BC20EAA
:101AE000C86FCB6BC80ECA6FCD6BCF0ECC6FCF6BF0
:101AF000D50ECE6FD16BDC0ED06FD36BE30ED26FF1
:101B0000D56BEA0ED46FD76BF20ED66FD96BFA0E87
:101B1000D86F010EDB6F020EDA6F010EDD6F0A0E59
:101B2000DC6F010EDF6F120EDE6F010EE16F1B0E18
:101B3000E06F010EE36F240EE26F010EE56F2E0ED3
:101B4000E46F010EE76F370EE66F010EE96F410E8D
:101B5000E86F010EEB6F4C0EEA6F010EED6F560E43
:101B6000EC6F010EEF6F610EEE6F010EF16F6C0EF8
:101B7000F06F010EF36F780EF26F010EF56F840EA9
:101B8000F46F010EF76F910EF66F010EF96F9D0E57
:101B9000F86F010EFB6FAB0EFA6F010EFD6FB80E02
:101BA000FC6F010EFF6FC60EFE6F010E0201016F8A
:101BB000D50E006F010E036FE40E026F010E056F6C
:101BC000F30E046F020E076F030E066F020E096F0D
:101BD000140E086F020E0B6F250E0A6F020E0D6FAA
:101BE000370E0C6F020E0F6F490E0E6F020E116F43
:101BF0005B0E106F020E136F6F0E126F020E156FD9
:101C0000830E146F020E176F970E166F020E196F68
:101C1000AC0E186F020E1B6FC20E1A6F020E1D6FF4
:101C2000D90E1C6F020E1F6FF00E1E6F030E216F78
:101C3000080E206F030E236F210E226F030E256FF7
:101C40003B0E246F030E276F550E266F030E296F70
:101C5000710E286F030E2B6F8D0E2A6F030E2D6FE2
:101C6000AA0E2C6F030E2F6FC80E2E6F030E316F4E
:101C7000E70E306F040E336F070E326F040E356FB0
:101C8000280E346F040E376F4A0E366F040E396F0C
:101C90006D0E386F040E3B6F910E3A6F040E3D6F60
:101CA000B70E3C6F040E3F6FDE0E3E6F050E416FA8
:101CB000406F436F2F0E426F050E456F590E446FF4
:101CC000050E476F850E466F050E496FB20E486FC1
:101CD000050E4B6FE10E4A6F060E4D6F110E4C6FE5
:101CE000060E4F6F430E4E6F060E516F760E506FFD
:101CF000060E536FAB0E526F060E556FE10E546F0A
:101D0000070E576F1A0E566F070E596F540E586F05
:101D1000070E5B6F900E5A6F070E5D6FCE0E5C6FF5
:101D2000080E5F6F0E0E5E6F080E616F500E606FD3
:101D3000080E636F940E626F080E656FDB0E646FA2
:101D4000090E676F230E666F090E696F6E0E686F5E
:101D5000090E6B6FBB0E6A6F0A0E6D6F0B0E6C6F08
:101D6000010E2B6E0001800E2B5C1DE201EE6EF069
:101D7000D8902B34E926000EEA22EECF06F0EFCF02
:101D800007F0D8900730036E0630026E01EE6EF059
:101D9000D8902B34E926000EEA2202C0EEFF03C0E1
:101DA000EFFF2B2ADFE312000101716B2E0E706F23
:101DB000736B310E726F756B320E746F776B330EFF
:101DC000766F796B350E786F7B6B360E7A6F7D6B25
:101DD000380E7C6F7F6B3A0E7E6F816B3B0E806F8F
:101DE000836B3D0E826F856B3F0E846F876B400E59
:101DF000866F896B420E886F8B6B440E8A6F8D6B7A
:101E0000460E8C6F8F6B480E8E6F916B4A0E906FE3
:101E1000936B4C0E926F956B4E0E946F976B510EA9
:101E2000966F996B530E986F9B6B550E9A6F9D6BC7
:101E3000580E9C6F9F6B5A0E9E6FA16B5D0EA06F2C
:101E4000A36B5F0EA26FA56B620EA46FA76B650EEE
:101E5000A66FA96B680EA86FAB6B6B0EAA6FAD6B0C
:101E60006E0EAC6FAF6B710EAE6FB16B740EB06F68
:101E7000B36B770EB26FB56B7B0EB46FB76B7E0E24
:101E8000B66FB96B820EB86FBB6B860EBA6FBD6B47
:101E9000890EBC6FBF6B8D0EBE6FC16B910EC06F94
:101EA000C36B950EC26FC56B9A0EC46FC76B9E0E47
:101EB000C66FC96BA20EC86FCB6BA70ECA6FCD6B76
:101EC000AC0ECC6FCF6BB10ECE6FD16BB60ED06FA8
:101ED000D36BBB0ED26FD56BC00ED46FD76BC60E53
:101EE000D66FD96BCB0ED86FDB6BD10EDA6FDD6B93
:101EF000D70EDC6FDF6BDD0EDE6FE16BE30EE06FA4
:101F0000E36BEA0EE26FE56BF10EE46FE76BF70E41
:101F1000E66FE96BFE0EE86F010EEB6F060EEA6FDF
:101F2000010EED6F0D0EEC6F010EEF6F150EEE6FE3
:101F3000010EF16F1D0EF06F010EF36F250EF26FA3
:101F4000010EF56F2D0EF46F010EF76F360EF66F62
:101F5000010EF96F3E0EF86F010EFB6F470EFA6F20
:101F6000010EFD6F510EFC6F010EFF6F5A0EFE6FDA
:101F7000010E0201016F640E006F010E036F6E0E01
:101F8000026F010E056F790E046F010E076F830E4D
:101F9000066F010E096F8E0E086F010E0B6F9A0E01
:101FA0000A6F010E0D6FA50E0C6F010E0F6FB10EB3
:101FB0000E6F010E116FBE0E106F010E136FCA0E61
:101FC000126F010E156FD70E146F010E176FE50E0D
:101FD000166F010E196FF30E186F020E1B6F010EB4
:101FE0001A6F020E1D6F0F0E1C6F020E1F6F1E0E5A
:101FF0001E6F020E216F2E0E206F020E236F3E0EFB
:10200000226F020E256F4E0E246F020E276F5F0E99
:10201000266F020E296F700E286F020E2B6F820E34
:102020002A6F020E2D6F940E2C6F020E2F6FA70ECB
:102030002E6F020E316FBA0E306F020E336FCE0E5E
:10204000326F020E356FE20E346F020E376FF70EED
:10205000366F030E396F0D0E386F030E3B6F230E74
:102060003A6F030E3D6F3A0E3C6F030E3F6F520EF8
:102070003E6F030E416F6A0E406F030E436F830E77
:10208000426F030E456F9C0E446F030E476FB60EF2
:10209000466F030E496FD10E486F030E4B6FED0E66
:1020A0004A6F040E4D6F0A0E4C6F040E4F6F270ED1
:1020B0004E6F040E516F450E506F040E536F640E39
:1020C000526F040E556F840E546F040E576FA50E99
:1020D000566F040E596FC70E586F040E5B6FEA0EF1
:1020E0005A6F050E5D6F0E0E5C6F050E5F6F320E40
:1020F0005E6F050E616F580E606F050E636F7F0E89
:10210000626F050E656FA70E646F050E676FD00EC8
:10211000666F050E696FFB0E686F060E6B6F260EFD
:102120006A6F060E6D6F530E6C6F010E2B6E000101
:10213000800E2B5C1DE201EE6EF0D8902B34E92668
:10214000000EEA22EECF06F0EFCF07F0D89007306E
:10215000036E0630026E01EE6EF0D8902B34E92645
:10216000000EEA2202C0EEFF03C0EFFF2B2ADFE3DE
:1021700012000101716B2D0E706F020E2B6E0001AB
:10218000800E2B5C37E22B04086E01EE6EF0D890C7
:102190000834E926000EEA22EECF06F0EFCF07F072
:1021A00006C010F007C011F00AEC01F013C017F0E0
:1021B00012C016F011C015F010C014F09A0E136E74
:1021C000990E126E3B0E116E830E106E29EC00F00C
:1021D000B7EC00F0026E11C003F001EE6EF0D89083
:1021E0002B34E926000EEA2202C0EEFF03C0EFFF07
:1021F0002B2AC5E3010E2B6E800E2B5C1DE201EE37
:102200006EF0D8902B34E926000EEA22EECF06F0CD
:10221000EFCF07F0D8900730036E0630026E01EE64
:102220006EF0D8902B34E926000EEA2202C0EEFFB1
:1022300003C0EFFF2B2AE0E312000101716B2C0EAB
:10224000706F736B2F0E726F756B310E746F776BCF
:10225000320E766F796B340E786F7B6B360E7A6F39
:102260007D6B380E7C6F7F6B390E7E6F816B3B0E02
:10227000806F836B3D0E826F856B3F0E846F876B23
:10228000420E866F896B440E886F8B6B460E8A6F89
:102290008D6B480E8C6F8F6B4B0E8E6F916B4D0E4E
:1022A000906F936B500E926F956B530E946F976B6C
:1022B000560E966F996B580E986F9B6B5B0E9A6FCC
:1022C0009D6B5F0E9C6F9F6B620E9E6FA16B650E88
:1022D000A06FA36B680EA26FA56B6C0EA46FA76BAB
:1022E000700EA66FA96B730EA86FAB6B770EAA6FFB
:1022F000AD6B7B0EAC6FAF6B7F0EAE6FB16B840EB0
:10230000B06FB36B880EB26FB56B8D0EB46FB76BD9
:10231000920EB66FB96B970EB86FBB6B9C0EBA6F0F
:10232000BD6BA10EBC6FBF6BA60EBE6FC16BAC0EBA
:10233000C06FC36BB20EC26FC56BB80EC46FC76BF4
:10234000BE0EC66FC96BC40EC86FCB6BCB0ECA6F07
:10235000CD6BD20ECC6FCF6BD90ECE6FD16BE00EA2
:10236000D06FD36BE80ED26FD56BF00ED46FD76BF6
:10237000F80ED66F010ED96FD86BDB6F090EDA6FCE
:10238000010EDD6F120EDC6F010EDF6F1B0EDE6FB4
:10239000010EE16F250EE06F010EE36F2F0EE26F6D
:1023A000010EE56F390EE46F010EE76F430EE66F25
:1023B000010EE96F4E0EE86F010EEB6F5A0EEA6FD9
:1023C000010EED6F650EEC6F010EEF6F710EEE6F8B
:1023D000010EF16F7E0EF06F010EF36F8B0EF26F38
:1023E000010EF56F980EF46F010EF76FA60EF66FE3
:1023F000010EF96FB40EF86F010EFB6FC30EFA6F8A
:10240000010EFD6FD20EFC6F010EFF6FE20EFE6F2C
:10241000010E0201016FF20E006F020E036F030E38
:10242000026F020E056F150E046F020E076F270E66
:10243000066F020E096F390E086F020E0B6F4C0EFD
:102440000A6F020E0D6F600E0C6F020E0F6F750E8D
:102450000E6F020E116F8A0E106F020E136FA00E18
:10246000126F020E156FB70E146F020E176FCE0E9D
:10247000166F020E196FE70E186F030E1B6F1A6BA3
:102480001D6F1A0E1C6F030E1F6F340E1E6F030E8E
:10249000216F500E206F030E236F6D0E226F030EFF
:1024A000256F8A0E246F030E276FA90E266F030E69
:1024B000296FC90E286F030E2B6FEA0E2A6F040EC8
:1024C0002D6F0B0E2C6F040E2F6F2E0E2E6F040E21
:1024D000316F530E306F040E336F780E326F040E6F
:1024E000356F9F0E346F040E376FC70E366F040EB4
:1024F000396FF00E386F050E3B6F1B0E3A6F050EED
:102500003D6F470E3C6F050E3F6F740E3E6F050E1C
:10251000416FA40E406F050E436FD50E426F060E3D
:10252000456F070E446F060E476F3B0E466F060E53
:10253000496F710E486F060E4B6FA90E4A6F060E5B
:102540004D6FE20E4C6F070E4F6F1E0E4E6F070E53
:10255000516F5C0E506F070E536F9B0E526F070E3C
:10256000556FDD0E546F080E576F210E566F080E13
:10257000596F670E586F080E5B6FB00E5A6F080EDA
:102580005D6FFB0E5C6F090E5F6F490E5E6F090E8B
:10259000616F990E606F090E636FED0E626F0A0E28
:1025A000656F420E646F0A0E676F9B0E666F0A0EB0
:1025B000696FF70E686F0B0E6B6F560E6A6F0B0E1E
:1025C0006D6FB80E6C6F010E2B6E0001800E2B5CD0
:1025D0001DE201EE6EF0D8902B34E926000EEA22BF
:1025E000EECF06F0EFCF07F0D8900730036E06303D
:1025F000026E01EE6EF0D8902B34E926000EEA222E
:1026000002C0EEFF03C0EFFF2B2ADFE312002B6AAC
:10261000300E2B5C08E2F36A03EE6EF02B50F3CF22
:10262000EBFF2B2AF5E37F0E03019E6F9F6F7E0E5B
:10263000A06FA16F7C0EA26F780EA36F720EA46FB5
:10264000700EA56FA66F600EA76F480EA86F400EA4
:10265000A96F9EC302F002C0AAF39FC302F002C09A
:10266000ABF3A0C302F002C0ACF3A1C302F002C0FE
:10267000ADF3A2C302F002C0AEF3A3C302F002C0E6
:10268000AFF3A4C302F002C0B0F3A5C302F002C0CE
:10269000B1F3A6C302F002C0B2F3A7C302F002C0B6
:1026A000B3F3A8C302F002C0B4F3A9C302F002C09E
:1026B000B5F3B66FB76B3E0EB86FB96F7C0EBA6FDD
:1026C000780EBB6F720EBC6F700EBD6FBE6F600E6A
:1026D000BF6F480EC06F400EC16FC26FC36B300E2C
:1026E000C46F7E0EC56F6C0EC66F580EC76F520E4C
:1026F000C86F700EC96F300ECA6F280ECB6F080EF0
:10270000CC6FD00ECD6F780ECE6FCF6B300ED06FFA
:102710007E0ED16F6C0ED26F580ED36F520ED46FE7
:10272000700ED56F300ED66F280ED76F6A0E2B6ED7
:102730000001800E2B5C08E2F36A03EE6EF02B5072
:0C274000F3CFEBFF2B2AF4E31200FFD7CD
:020000040030CA
:0300010006160ED2
:020005008580F4
:060008000FC00FE00F40E5
:00000001FF
